:020000040000FA
:060000000219FD0200C818
:03000B0002008D63
:03002B000200923E
:03005B000202CBD3
:030073000200B5D3
:100080000406080C10182030406080A0C0C28D0506
:100090004032C0D0C0E0C2CF0541E5646009E563ED
:1000A000600575630001B0756301E52360021523E7
:1000B000D0E0D0D032C2AF53E67F7592FA7593FF8D
:1000C000C22053917FD2AF32C2AF53E6EFC0D0C04F
:1000D000E0C0F0D2D3D2AF5388EFA88AA98CAA404F
:1000E000308D010A758A00758C00754000438810B8
:1000F000E564700AC3E833F8E933F9EA33FA3033D8
:100100001FE8C4540FFAE9C454F04AFAC3132AFA98
:10011000C3E833F8E933F9E82AFAE93406FB217336
:1001200030320FC3E833E933FAE82AFAE93400FB46
:100130002173303115E875F056A4AAF0E975F05630
:10014000A42AFAC5F03400FB2173C3EA13FAE913B9
:10015000F9E813F8E875F056A4AAF0E975F056A48A
:100160002AFAC5F03400C313FBEA13FAC3EB13FBFE
:10017000EA13FAC3EB94125006C3EB9406501A0527
:1001800022E52270021522C3E522940A500241BEE4
:100190007552007A007B00418CE522600215223006
:1001A00035067C007D0821B3AC31AD32303A04AC69
:1001B00033AD34C3EA9CFAEB9DFB9208AE5EAF5FB1
:1001C000303A425007203409D23421D1303402C2AF
:1001D00034303404AE60AF61203902B234C3EA3344
:1001E000FAEB33FBA208500AEAF42401FAEBF434E8
:1001F00000FBC3EA9450FAEB9400FB501478007AA9
:10020000007B004111A208500878007A007B004171
:1002100070E5255403601B202A18E55B33F9EB7069
:1002200007C3E99A4002E9FAE53CC4332AFAEB3401
:1002300000FBEA8EF0A4F9AAF0EB8EF0A42AFAC52E
:10024000F03400FBC3EB13FDEA13F8C3ED13FDE834
:1002500013F80FEF146004C3E833F8C3E933EA334B
:10026000FAEB33FBDFEDEB30E30678FF7AFF7B0739
:100270008852D230C3E559FC955A4002AC5AC3ECBF
:1002800095525008EC75F008A4FAABF0EAF4F8EBDC
:10029000F45407F9C3E89428FAE99400FB50047A6F
:1002A000007B00885489558A568B5775230AD0F0F5
:1002B000D0E0D0D053F7DF43F74043E61032752348
:1002C0000AD0F0D0E0D0D043E61032C2AF53A8FE3F
:1002D000C0D0C0E0D2D3A8F9E55830E20AE5FA2050
:1002E000E24220E13F41EFE5FA30E23820E135C358
:1002F000E55513F8E55413F5FB88FCC3E55713F8EF
:10030000E55613F5E988EA85555853F7BFC3E5521A
:10031000940140057553006124E5532401F55350C1
:10032000037553FF53F7DFD0E0D0D043A801D2AF1D
:10033000327901801479038010790A800C791E804B
:10034000087964800479C880007817E4D5E0FDD886
:10035000FAD9F6227A147B7880127A107B8C800C82
:100360007A0D7BB480067A0B7BC88000E562D5E00D
:1003700001227902E4C293D5E0FDD292D5E0FDC21C
:1003800092D5E0FDD293D5E0FDE920E002D2903095
:10039000E002D294E562D5E0FDE920E002C29030AF
:1003A000E002C2947496D5E0FDD9C9EAF8D5E0FD23
:1003B000D8FBDBB8C2932278FF20282879A1E76018
:1003C00023E548601F74FF8548F084853FF030299D
:1003D0000375F005A4F8C5F0600278FFC3E8955BEB
:1003E0005002A85B885A22C3E54794A0E5489400D0
:1003F000E55A50031461F8046002F55A2275E8903A
:1004000022055CC3E55C9408405330EDF4A8BDA917
:10041000BE755C00E9FA79A0E76041EA7006E55D27
:100420006018800CC3E8955D600EE55D5005600ABC
:100430001480070460FA8002E55DF55DC3956740AE
:100440001B7559C0C394044013755980C39404406C
:100450000B755940C39404400375590022E5592493
:1004600010500274FFF55922743279A687F0A4C5A2
:10047000F0A2F733F8C3E895594002A859885B22E7
:100480007547007548F022C2AF75C800A8CCA9CD49
:10049000AA4130CF010A75C804D2AFC3EA13FAE902
:1004A00013F9E813F8AB42AC4388428943C3E89B95
:1004B000F8E99C20280A547FF9302C02A1A481FE7F
:1004C000AD448A44F9EA9D547FFA600478FF79FFCD
:1004D000AE45AF468B458C46A842A943C3E89EF87B
:1004E000E99FF9C3E54813FBE54713FAE82AF54706
:1004F000E93BF54850067547FF7548FFA14BAA47F1
:10050000AB48AC47AD487E047F02C3EB9404400D7A
:100510001E1FC3EB940840052029021E1FC3ED13C4
:10052000FDEC13FCDEF7C3EA9CFAEB9DFBEF6009E0
:10053000C3E913F9E813F8DFF7EA28FAEB39FB8A85
:10054000478B4850067BFF8B478B48C3EB94025088
:1005500002D22C3028047F03A1767892E6FFC3E50F
:100560003D948240110FC3E53D94A040010FC3EFBD
:10057000940640027F057E02E548C4540FF9E54821
:10058000C454F0F8E547C4540F28F8C3E89EFAE9CC
:100590009400FB4009C3EA9401EB940050047A01F3
:1005A000E4FBA1F0AA47AB48EBC4FEEAC4540F4EEB
:1005B000FCC3EA9CFAEB9400FBC3E813C313F8EA0C
:1005C00028FAEB3400FB8A478B48C3EB94024002C5
:1005D000C22C7802EBC4FE7B00EAC4540F4EFAC36F
:1005E000EA98FA4005C3940150027A017892E6FF36
:1005F000302002A1F0854E92854F93D22043E680B1
:10060000C3E49AF8E49BF9C3E833F8E933F9302CF2
:1006100002C182E8FAE9FBD3E913FDE813FC884E36
:10062000894FC3EF94036037EF20E00CE82CF8E922
:100630003DF9ECFAEDFB8013E828F8E939F9C3E855
:100640002401F8E93400F97AFF7BFFC3EF940340FB
:100650000E8A508B51884A894B8C4C8D4DC1B6887F
:100660005089518A4A8B4B8C4C8D4D3028127550D5
:10067000F07551FF754CF0754DFF754EF0754FFFDD
:10068000C1B6E8FAD3E813FC884EC3EF94036020A8
:10069000EF20E007E82CF8ECFAC1A2E8282401F8E2
:1006A0007AFFC3EF940340088A50884A8C4CC1B645
:1006B00088508A4A8C4C302002C1B6753A02D2204A
:1006C00043E680E5255403602DA847A948C3E913F4
:1006D000F9E813F8302804E92440F9C2AF53E67F63
:1006E000759100C3E498F594E499F595759104D259
:1006F0002043E680D2AF22D2217549007520003018
:100700002B03752040800ED22175490075204030A2
:100710002B0375200078017901202C20E525540356
:100720006002C2217914E548C313700104F8C39430
:100730001440027814302804781B791BC3E833F87E
:10074000C3E933F9202010E549600C302803D53A7D
:1007500004D223E1CBD1BE0549E59B5440B520022C
:10076000E1B530280908C3E899400118E144202187
:100770000A08C3E8994002E115E144C221C2AF531F
:10078000E67F759100302C127594007595F0759187
:1007900004D22043E680D2AFE115E5487EFFC333A3
:1007A0004009C3334005C3334001FEC3E49E759442
:1007B00000F595E18EC3E53994015002E115302131
:1007C00002E115D802E1C9E144C223C2AF53E67F7A
:1007D000759100855094855195759104854A92854F
:1007E0004B93D22043E680D2AFE525540360072027
:1007F00029020539801030230D202B0A20210715EE
:10080000811581020F282278003021027801E53D10
:1008100075F007A4F9E5F028F5F0E9A2F013A2F1CC
:1008200013A2F213F53DC394785003753D78C3E5E8
:100830003D953E400BD222C290C292C29475D57FA4
:100840003020020140854C92854D93D22043E680B2
:1008500022203810C2AFC293D29175D54FD2AF7556
:100860009F202125C2AFC293D29575D57CD2AF759A
:100870009F202125203811C2AFC29475D573D29123
:10088000D2AF759F30020925C2AFC29075D573D221
:1008900095D2AF759F10020925203810C2AFC291C2
:1008A000D29575D573D2AF759F108079C2AFC295BE
:1008B000D29175D573D2AF759F308069203811C23F
:1008C000AFC29275D57CD295D2AF759F2002092513
:1008D000C2AFC29275D54FD291D2AF759F20020997
:1008E00025203810C2AFC295D29375D57CD2AF7592
:1008F0009F308031C2AFC291D29375D54FD2AF75C0
:100900009F108021203810C2AFC29075D54FD2936E
:10091000D2AF759F10800EC2AFC29475D57CD293B2
:10092000D2AF759F30C22222C290C292C294C291AD
:10093000C293C29575D57F22788076FF0876FF082E
:1009400076FF0876FF0876FF0876FF0876090876B6
:10095000FF087601788C76010876FF0876FF087626
:10096000FF0876FF0876FF0876030876FF0876FF13
:100970000876FF0876250876D0087628087650088D
:1009800076040876FF0876020876FF08767A0876FD
:10099000FF0876070876010876FF0876FF087600DC
:1009A00008760022FA75F00CA4ABF0EAC333F874B1
:1009B0000133F9E8C333F8E933F9E8C32BF8E93434
:1009C00000F9E8C333F8E933F9227888E6C39403E1
:1009D000D23A5002C23AC238E630E102D238A238E6
:1009E00092397886E6149000809378A6F67886E6A9
:1009F000F53FC394025003753F02789CE6753EFFB5
:100A0000B40203753EA0B40303753E8278A0E6F8F5
:100A1000600674282409D8FCF5677896E631A48826
:100A2000318932789EE631A4883389347897E6316B
:100A3000A4883589363128223035117A007B007C34
:100A4000FF7D007E00519F8B5F8A5E22303A2278C4
:100A500096E6FA7B00789EE6FC7D00C3EA33FAEB6B
:100A600033FBC3EC33FCED33FD7E0A519F8B618A6F
:100A7000607896303A02789EE6FA7B007897E6FC3A
:100A80007D007E00303A10C3EA33FAEB33FBC3EC4F
:100A900033FCED33FD7E0A519F8B5F8A5E2222C3B9
:100AA000EC9EFCED9400FDC3EC9AFCED9BFDC3ECC9
:100AB0009423ED940050047C237D00C3EC94FFED5F
:100AC000940140047CFF7D017BFF0B7A000AEA70F1
:100AD00009C3EC33FCED33FD41CAEC8AF0A4AEF05F
:100AE000ED8AF0A42E947C40E4EAF460DD22D23555
:100AF000513812033D12033D7A007B007C10120333
:100B000035E5522AFA74003BFBDCF37C04C3EB139B
:100B1000FBEA13FADCF7FFEB60027FFFC2355138C6
:100B20002278A5E6F95403D2867002C286E9540CF5
:100B3000D2877002C287E95430D2967002C296E919
:100B400054C07000227565007566007597DE759754
:100B5000AD7581C043FF8075EF0675A9003128751A
:100B6000803F75F1F075A4C075803F75D4FF759016
:100B70000075F27F75A57F75900075D57F75A6010C
:100B800075E34075E202C290C292C294120341D250
:100B900091D293D295120331C291C293C29531285A
:100BA000E4F8F6D8FD3138F169789886627530013D
:100BB000C2AF12034512035412033D12035A12032B
:100BC0003D12036012033D7121C2AF756500756669
:100BD0000078FA79FA308507D9FBD8F7021C003182
:100BE000CA513878988662312875A91375A710758F
:100BF000C10075A70075640075E405758811758ED0
:100C00000475890975C80475910475D84075D908AB
:100C100075F782759E0375960275DA4275DB42752B
:100C2000A82375E69075F310759B80759D0075D1AE
:100C30000C75BCB975BB1075E88075B20112033133
:100C4000D2AF753C00C230120345C231752200128A
:100C50000341C3E522940A4024D231C232752200F6
:100C6000120341C3E522940A4013D232C2337522E3
:100C700000120341C3E522940A4002D23312033525
:100C8000203003020BC9C2AF1203541203541203E3
:100C900054D2AF120345303A02A13B120335788C8F
:100CA000E6C394015002A13BE530C394015002A178
:100CB0003B7565A57566F17F02D235513812034147
:100CC000C2AFC2355138C3E552947FD2AF406C12E7
:100CD0000331C2AF120366D2AFDFDE51EEC3EF784D
:100CE00097F61203451210517F0AD235513812037C
:100CF00041C2AFC2355138C3E552947FD2AF50E8FC
:100D0000120331C2AF120354120339120354D2AF8B
:100D1000DFD851EEEF24037896F6F87997E7C3947D
:100D2000234003985006E824237897F6120345F1F0
:100D3000A3121080120341513861C97565007566B0
:100D4000001203417801303A027805C3E552984019
:100D5000028196C2AF120366120366120366D2AF17
:100D6000120345753000E4F537F5380537E537F4FB
:100D7000703E0538789AE67819146012783214605B
:100D80000D787D14600878FA146003753800C3E5A7
:100D90003898401C3128120331153875370078997E
:100DA0008662C2AF120366D2AF78988662120341A0
:100DB000120339E523700261C97801C3E5529840F6
:100DC000AA120341E5237003020BC9C2AF3128E424
:100DD000D2AFE4F55CF524F525F53D755C0812030A
:100DE000311203FD30EDFDA8BDA9BEE97001F88800
:100DF0005D120401755C08C2AF7559FF1204688565
:100E00005B59855B5AD2AF75A71075C13075A700C5
:100E100075A903756401303A07C238303402D238FC
:100E2000D22875390011E1310412048012048712AE
:100E3000048012048712048012070711071151124F
:100E400004871206F7202C031203B7302C03120379
:100E5000E71107117412048712070711071199127D
:100E600004871206F7110711BC1204871207071135
:100E70000711E11204871203FD1206F7110731046E
:100E8000120401120487302827855B5979187A0CDF
:100E9000C3E53999400EC228D2298A3B855B598522
:100EA0005B5A800CC3E55294014003020E38E130D6
:100EB00030291C202B19E53B147006C229D22AC107
:100EC00038F53BC3E55294014003020E388061754A
:100ED0003C0078FA79A4E760027803C3E5539850A0
:100EE0004FE523604B303A17203805203407800F38
:100EF000303402800A202B07D22B855B59C16278DF
:100F0000F0302B05855B597820C3E54898500302E3
:100F10000E38302B1BC22BC238303402D238D229C3
:100F2000753B12855B59C138053CE5526002E133DF
:100F3000753C00C2AF312875240075250075A913D2
:100F400075A71075C10075A700756400D2AF1203B4
:100F500041312878A4E66006D291D293D295C3E5B8
:100F60003C9404400261C9A166901A0D7820F1E01A
:100F7000E520B4550AA3F1E0E520B4AA02800631C9
:100F800038F1A3801D901A0378807B0AF1E0A30852
:100F9000DBFA901A0F788C7B1AF1E0A308DBFA9049
:100FA0001A2922C2AF121025121000901A007410D4
:100FB000F1E5A37403F1E5A37421F1E5901A037838
:100FC000807B0AF1E4A308DBFA901A0F788C7B1A75
:100FD000F1E4A308DBFA121039121014901A292236
:100FE000E493F622E6438F01538FFDFFC3E583941C
:100FF0001C400122EF8565B78566B7F0538FFE224E
:10100000438F02438F018565B78566B7901A0DF04F
:10101000538FFC22901A0D7455120FE5901A0E741E
:10102000AA120FE5227A3079D07820901A40120F58
:10103000E0E520F709A3DAF6227A3079D0901A4059
:10104000E7120FE509A3DAF8227C05120345DCFB61
:1010500022C2AF12035412035A1203601203661223
:10106000033912035412035A120360120366120367
:101070003912035412035A120360120366D2AF22CC
:10108000C2AF12036612036012035A120354120312
:101090003912036612036012035A12035412033901
:0F10A00012036612036012035A120354D2AF22D6
:1019FD00020B45100321FFFFFFFFFFFF09FF01FF52
:101A0D0055AA01FFFFFFFFFF03FFFFFF25D0285061
:0D1A1D0004FF02FF7AFF0701FFFF0000FF3A
:101A400023455F485F3230232020202020202020A3
:101A500023424C48454C492445464D3842323123B7
:101A60002020202020202020202020202020202076
:101C0000C2AFC2D37597DE7597AD7581C075A90057
:101C100043FF80752438752503B1DB7529A5752A26
:101C2000F143F12053A4DFD28575D4FF75E3407DE5
:101C3000FA780379E67C10752200752300901DE880
:101C40007B0675249875250130850281482085081A
:101C5000D8FBD9F9DCF781BA308508D8FBD9F9DC93
:101C6000F781BAB19BE493A3C39A6004DDC381BA40
:101C7000DBDBB18D600281317B08E493FAA3B16EA6
:101C8000DBF87A30B16E752200752300B18DEAFC65
:101C9000EBFDC3ED94FE400EB18D8A278B28ED300D
:101CA000E0048A828B83B18D7AC270D8C3ED94FE32
:101CB000601950CEBD0029EC600F7520007521FF22
:101CC000752900752A000200008100A827A92808AC
:101CD00009D804D90281DDB191EAF281D10D81A642
:101CE000C3ED94035051EDA2E092007AC5C3E582A2
:101CF0009400E583941C508C200010438F02438F86
:101D0000018529B7852AB7F0300027A827A9280818
:101D100009438F01538FFDD804D902A132C3E58353
:101D2000941C4003A3A117E28529B7852AB7F0A325
:101D3000A117538FFC81827AC1BD030CE493A3FAEF
:101D4000B152DCF8B14A81828184AA22AB23B16E00
:101D5000EBFAEA6222752608C3E52313F523E52290
:101D600013F52250066323A0632201D526EAB1DBD6
:101D7000B1DB75260AEAF4200102D285300102C2E5
:101D800085B1DBC3134002C201D526EB22B191EA33
:101D9000FB208502A191308502A196752608AE240C
:101DA000AF25C3EF13FFEE13FEB1DFB1DBC3EA13C0
:101DB0003085024480FA30E703632201C3E5231330
:101DC000F523E52213F52250066323A0632201D5F3
:101DD00026D9E52265236523F52222AE24AF250E00
:101DE0000FDEFEDFFCD20122424C48656C693437BD
:061DF0003163E8B20601B8
:00000001FF
